:103D43000FA60FA00F990F920F8B0F840F7C0F7488
:103D53000F6B0F620F580F4E0F430F380F2C0F1FAF
:103D63000F120F050EF70EE80ED80EC80EB70EA5EC
:103D73000E930E800E6C0E580E420E2C0E150DFD7A
:103D83000DE40DCB0DB10D950D790D5D0D3F0D209E
:103D93000D010CE10CC00C9E0C7C0C590C350C1065
:103DA3000BEA0BC40B9E0B760B4F0B260AFD0AD4B2
:103DB3000AAA0A800A550A2A09FF09D409A8097C14
:103DC3000950092508F908CD08A10875084A081EF5
:103DD30007F307C8079D07730749072006F706CEB1
:103DE30006A6067E06570630060A05E405BF059BB0
:103DF300057705540532051004EF04CE04AE048F95
:103E0300047104530435041903FD03E203C703AD2E
:103E13000394037B0363034B0334031E030802F37E
:103E230002DE02CA02B602A30291027F026D025CA5
:103E3300024C023C022C021D020E020001F201E4BC
:103E430001D701CA01BE01B101A6019A018F018503
:103E5300017A01700166015D0153014A0141013993
:103E630001310129012101190112010B010400FD96
:103E730000F700F000EA00E400DE00D900D300CE32
:103E830000C900C400BF00BA00B500B100AD00A86E
:103E930000A400A0009C009900950091008E008A68
:103EA300008700840081007E007B00010C01010477
:103EB30002011E030A960401320503030600640788
:103EC300010108000009015A0E01010F000112004F
:103ED3006413010114013C1501FA1664FA17FFFF7C
:103EE3001D00072000072400022701012F013C3099
:103EF300010132010335FFFF3603073CFFFF3DFF9E
:103F0300FF180002191E461A00021B00022D32C8B8
:103F13002E0001FAFAFA18000019FFFF1A00001B1D
:103F230000002D32C82E0001FAFAFA18000019FF1A
:103F3300FF1A00001B00002DFFFF2EFFFFFAFAFA05
:10004800900786E0FEA3E0FF7457BE0010D39F40E0
:100058000C903EAD12001EE493F599804C9000146C
:10006800E0D394044014900786E0FEA3E0FF903E9E
:10007800AD12001EE493F599802F900014E0D394FC
:10008800034014900786E0FEA3E0FF903EC21200F2
:100098001EE493F5998012900786E0FEA3E0FF9096
:1000A8003ED712001EE493F59990078612000E9031
:1000B8000786E0FEA3E0FF746C6F4E7003751300B3
:1000C80022900072E0B401087402900072F0D20C21
:1000D80090013AE090002AF090013BE090002BF06C
:1000E80090013CE090002CF0A20AB3401690013A2F
:1000F800E0700C90013BE0700690013CE0600280EB
:1001080002C20A90013AE0B4300F90013BE0B447D4
:100118000890013CE0643B60028004D20B8002C27C
:100128000BE558B40102800302024B900057E0F53A
:1001380066900062E0F568900063E0F569900074ED
:10014800E0F56A90007AE0900029F090007CE0F5F4
:100158006590007DE0F567900080E0F5649000818F
:10016800E0F563900090E0900041F0900091E090FD
:100178000042F0900092E0900043F0900093E090ED
:100188000044F0900094E0900045F0900095E090D5
:100198000046F0900096E0900047F0900097E090BD
:1001A8000048F0900099E0900033F090009AE090B9
:1001B8000034F090009BE0900035F090009CE090B7
:1001C8000036F0900079E0B4011790000A740FF03F
:1001D800A374FFF090000CE4F0A3F074029000798F
:1001E800F0900079E0B4035990000CE0FEA3E0FF22
:1001F80090000AE0FCA3E0FD12000374101240A373
:100208007408124095EF900026F0EF700674FF9086
:100218000026F07400900079F090000BE090002721
:10022800F090000AE0900028F0900026E0900789FE
:10023800F0900027E090078AF0900028E090078B64
:10024800F0803F900081E07006755801756300A248
:100258000AB3402E90013AE090002AF090013BE06A
:1002680090002BF090013CE090002CF090002AE0E8
:10027800700C90002BE0700690002CE06002800269
:10028800C20AE5667003756602E568700375680260
:100298007E837FC2E5668E048F05FF1240858C3908
:1002A8008D3AE56975F0FAA4FFAEF0E5688E048F23
:1002B80005FF1240858C3D8D3E90004FE0F5609023
:1002C800004DE0FE900069E0B5061890004CE0FE95
:1002D800900068E0B5060C90004BE0FE900059E0F5
:1002E8006E606F900069E07006900068E0600674C8
:1002F80000900059F0900069E0B402089000497439
:1003080001F08005900049E4F0900068E0B402082C
:1003180090004A7401F0800590004AE4F09000686B
:10032800E0600690004AE060028005756003800383
:10033800756004E559B55802D20C900068E0900049
:100348004CF0900069E090004DF0900059E090006A
:100358004BF0740190009EF0740090009FF07400C0
:100368009000A0F074009000A1F074009000A2F03A
:1003780074009000A3F074009000A4F07401900041
:10038800A5F074009000A6F074009000A7F0740027
:100398009000A8F074009000A9F074009000AAF0F2
:1003A80074009000ABF074019000ACF07400900001
:1003B800ADF074009000AEF074009000AFF07400DF
:1003C8009000B0F074009000B1F074009000B2F0AA
:1003D8007401900362F07400900363F0740090035A
:1003E80064F07400900365F07400900366F0740084
:1003F800900367F07400900368F074009003A2F013
:1004080074009003A3F074009003A4F074009003A8
:10041800A5F074009003A6F074009003A7F0740090
:100428009003A8F074009003E2F074019003E3F0E5
:1004380074009003E4F074009003E5F074009003F6
:10044800E6F074009003E7F074009003E8F074019C
:10045800900422F07401900423F07400900424F0B6
:100468007400900425F07400900426F07400900441
:1004780027F07400900428F022E5B554F7F5B5E5A7
:10048800B554FDF5B5C292C291C290C207E5B55404
:10049800FBF5B5755104E55104F55290004FE0F5B0
:1004A80060900025E4F0C209E5B554FEF5B5C28EAA
:1004B800758D00758B00754C00752600752500D26A
:1004C8008E22750A00750900AE09AF0A7457BE007E
:1004D800039F5003020587903EAD12001EE49390DF
:1004E800004E1240BB0FBF00010EE0FC903EAD1263
:1004F800001EECFEE493FFEEC39F5026AE09AF0A40
:100508000FBF00010E903EAD12001EAE09AF0AE407
:1005180093FC903EAD12001EE49390004E1240BB37
:10052800ECF0AE09AF0A903EAD12001EE4939000C5
:100538004E1240BBE0FC903EAF12001EECFCE49370
:10054800FDECD39D4019903EAF12001EE493FC9041
:100558003EAD12001EE49390004E1240BBECF0AE8C
:1005680009AF0A74022FFF50010E8E098F0A780A0C
:10057800740126F6500418E436F640030204D0222B
:10058800750A00750900AE09AF0A7415BE00039F0D
:100598005003020655903F0412001EE49390004E4B
:1005A8001240BB0FBF00010EE0FC903F0412001E7A
:1005B800ECFEE493FFEEC39F5026AE09AF0A0FBFCF
:1005C80000010E903F0412001EAE09AF0AE493FC2E
:1005D800903F0412001EE49390004E1240BBECF0D2
:1005E800AE09AF0A903F0412001EE49390004E1229
:1005F80040BBE0FC903F0612001EECFCE493FDECCF
:10060800D39D4019903F0612001EE493FC903F04CE
:1006180012001EE49390004E1240BBECF0AE09AFFE
:100628000A740F6F4E7006750A15750900AE09AF8A
:100638000A74022FFF50010E8E098F0A780A74017E
:1006480026F6500418E436F6400302058E22750A91
:1006580000750900AE09AF0A7415BE00039F500368
:10066800020723903F1912001EE49390004E124097
:10067800BB0FBF00010EE0FC903F1912001EECFEFC
:10068800E493FFEEC39F5026AE09AF0A0FBF0001E7
:100698000E903F1912001EAE09AF0AE493FC903F7A
:1006A8001912001EE49390004E1240BBECF0AE0904
:1006B800AF0A903F1912001EE49390004E1240BBFF
:1006C800E0FC903F1B12001EECFCE493FDECD39D74
:1006D8004019903F1B12001EE493FC903F19120032
:1006E8001EE49390004E1240BBECF0AE09AF0A74C2
:1006F8000F6F4E7006750A15750900AE09AF0A74BA
:10070800022FFF50010E8E098F0A780A740126F60F
:10071800500418E436F6400302065C22750A007598
:100728000900AE09AF0A7415BE00039F5003020703
:10073800F1903F2E12001EE49390004E1240BB0F22
:10074800BF00010EE0FC903F2E12001EECFEE49369
:10075800FFEEC39F5026AE09AF0A0FBF00010E90EF
:100768003F2E12001EAE09AF0AE493FC903F2E12F2
:10077800001EE49390004E1240BBECF0AE09AF0AA5
:10078800903F2E12001EE49390004E1240BBE0FCF6
:10079800903F3012001EECFCE493FDECD39D401911
:1007A800903F3012001EE493FC903F2E12001EE48E
:1007B8009390004E1240BBECF0AE09AF0A740F6F75
:1007C8004E7006750A15750900AE09AF0A74022F36
:1007D800FF50010E8E098F0A780A740126F650041C
:1007E80018E436F6400302072A22054D22054C225A
:1007F800054EC2CF2290F800E4936406600280FEA2
:1008080075840175A70075FF80900788E4F075C9A5
:100818001075A70F75A1C775A70075D90075CEFF0C
:1008280075A70F75F1FE75F2FF75F33775F47875D6
:10083800A4BA75A5FF75A60775AE0075AFFF75D488
:100848008175D5FF75D6FF75D7FFC293C294C2874D
:10085800C2A1E5B554BFF5B5E5B554DFF5B5E5B5C5
:1008680054EFF5B5E5B5547FF5B5E5B554F7F5B5ED
:10087800E5B554FDF5B575A70075A20175A14775D5
:10088800F80975BC0175BE0475BD6C75BE0775BDEC
:10089800A075BE0875BD0175BC0075BB1875BC2078
:1008A80075BA0875E88075D11375A70F75E10575D8
:1008B800E20075C740759700759780740A124075F5
:1008C8007597C0E5975420700280F8758F0275A758
:1008D80000D2AF75980075A90C75A70F75AB437555
:1008E800ADFB75AC1E75A700758911758E00758CEA
:1008F80000758A00D2A9D28C758D00758B00D2AB99
:10090800D28E75CD0075CC0075CA0075CB00D2ADFE
:10091800C2CFD2CA7591047592007593CD75EF0652
:1009280075D94075CF01900786E4F0A3F0751300E0
:10093800751400C299D20AC20D12048174C8F51840
:1009480075170012267275A70FE5FB90001AF0E5DF
:10095800FA90001BF0E5F990001CF075A70090F8DC
:1009680000E493F5081227A9122CE3900789E09078
:100978000026F090078AE0900027F090078BE0901F
:100988000028F090078CE0900029F090078DE0F5A2
:100998006690078EE0F56890078FE0F569900790FC
:1009A800E0F56A900791E0F565900792E0F56790A9
:1009B8000793E0F564900794E0F563900795E0905D
:1009C800002AF0900796E090002BF0900797E090AF
:1009D800002CF0900798E0900041F0900799E09083
:1009E8000042F090079AE0900043F090079BE09057
:1009F8000044F090079CE0900045F090079DE0903F
:100A08000046F090079EE0900047F090079FE09026
:100A18000048F09007A0E0900033F09007A1E09024
:100A28000034F09007A2E0900035F09007A3E09022
:100A38000036F07400900082F090013AE0700C905B
:100A4800013BE0700690013CE060028004C20A802D
:100A580002D20A90F807E493900021F0900021E078
:100A6800440A900021F0900021E054FE900021F00B
:100A78007406900012F07402900013F090F802E4EB
:100A880093900014F07403900015F074039000160E
:100A9800F0740C900017F07405900018F090001492
:100AA800E0B404067404900018F0900014E0B40355
:100AB800067403900018F07405900019F090F8047B
:100AC800E49390001DF0740090001EF090F805E487
:100AD8009390001FF090F806E493900020F074FFC4
:100AE800900022F07446900125F0746F900126F072
:100AF8007472900127F07464900128F074209001BA
:100B080029F0744190012AF0744F90012BF074443D
:100B180090012CF0744590012DF0742090012EF076
:100B2800742090012FF07434900130F074539001C8
:100B380031F07450900132F07444900133F0900019
:100B48007AE0D394014006740090007AF075580159
:100B5800755901740390004CF01200C91204CA9030
:100B68000014E0B404051206568011900014E0D376
:100B780094044005120588800312072412269EE576
:100B8800B554FEF5B5900025E4F0900786E4F0A38F
:100B9800F0752400752300754800752A0075290032
:100BA800754900753200753100754A007554007535
:100BB8005500755A0075510475520175343C7533EA
:100BC80000757000756F007571CD7556007557000A
:100BD800754300754400754500754600755B0075E2
:100BE8004700754200754100900006E4F0A3F090BC
:100BF8000008E4F0A3F0755E00755F0090000E74C5
:100C0800FDF0A374E8F0900023E4F07464900024ED
:100C1800F0C200D201C202D203754D00756D00C248
:100C280097C2A0C296C295C2A2C20C7E017F009054
:100C38000028E01240A3900027E02FFF50010E90FB
:100C4800000AEEF0A3EFF0900026E0700674FF9023
:100C58000026F090000AE0FEA3E0FFEFD394FFEE39
:100C6800940F400790000AE4F0A3F074009000711C
:100C7800F07400900079F07400900082F074009095
:100C8800008DF074009000B4F0E567700375670498
:100C9800743A90074EF074FD90074FF09003D4E03B
:100CA800900414F0D2B0D2B7D2A7D2A6D2B1D2A3B0
:100CB800C207A2B6B39204A2B3B39205D29CD2ECF7
:100CC80075CF01A298B34005C298123047E513606A
:100CD80006A299B3B340028005C2991235B7E5144C
:100CE80064016005E514B4040280D5E54DD394058C
:100CF800400CE55AC394C85002055A754D00E57179
:100D0800C394F0501A786F12003FAE6FAF70EFD3F4
:100D180094E8EE940340080571757000756F00C281
:100D28008E7E047F00E54C1240A3E58D75F004A487
:100D3800FDACF0EF2DFDEE3CFCE58B75F04084FF3B
:100D48007E00ED2FFFEC3EFE8E258F26D28EA2B6BA
:100D5800300401B35003020E9BA2B6300401B35015
:100D680003020E9BA2B640670554A20D400575FF0D
:100D7800A0D20DE5B54401F5B5900024E4F0E554A2
:100D8800D3956640487C837DC2AE25AF26123F438B
:100D98008E238F24E5482FFF50010E7401124095D1
:100DA8008E238F24852448755401C28E758D007555
:100DB8008B00754C00D28E7403BE00039F500690C2
:100DC80000257401F0E543B40603754300D204A27C
:100DD800B6B35003020E9BC20490006BE060181279
:100DE80036F8A200B34008E5B54408F5B58006E535
:100DF800B554F7F5B58002C20090006EE060181295
:100E0800384DA202B34008E5B54402F5B58006E5C1
:100E1800B554FDF5B58006E5B554FDF5B5A207B3A3
:100E28004004D2968002C296900059E06004D295A0
:100E38008002C29590004AE0B40104D2978002C2B1
:100E480097900049E0B40104D2A08002C2A0A20990
:100E5800B34004D2A28002C2A2900018E0FE900023
:100E680014E0C39E4009900014E0D394084009742C
:100E7800FB900023F012048190001DE060159000A3
:100E88001DE0FE900017E06E600974FE900023F0EC
:100E9800120481C2CA7E017F00E54E1240A3E5CD4F
:100EA8002FFF50010E8E278F28D2CAE565B401485E
:100EB80090000EE0FCA3E0FDEFC39DEE9C4039B22C
:100EC80008E52A45296013A208B34008E5B544049B
:100ED800F5B58006E5B554FBF5B590000EE0FEA328
:100EE800E0FF900010E0FCA3E0FDEF2DFDEE3CFCE0
:100EF80090000EECF0A3EDF0A2B3300501B350035F
:100F0800020FE9A2B3300501B35003020FE9A2B3FF
:100F18005003020FE20555A20D400575FFA0D20D42
:100F2800E5B54401F5B5900024E4F0E555D395689E
:100F38005003020FE07CEA7D60AE27AF28123F43E2
:100F48008E298F2AE5691240A374FF8E048F05FF4E
:100F58001240858C298D2AE5492DFD50010C74011C
:100F68008C068D071240958E298F2A852A49A20959
:100F7800B3401574641240A3900067E08E048F0597
:100F8800FF1240858C298D2A75550190000EE0FED0
:100F9800A3E0FFAC27AD2812000390000EEEF0A3EB
:100FA800EFF0E567FF124085740AFF124085900054
:100FB8007BE08C068D071240A374148E048F05FF06
:100FC800124085900010ECF0A3EDF0C2CA75CD0078
:100FD80075CC00754E00D2CAD205A2B3B34002C286
:100FE80005900025E0B40107E556C39406400302C6
:100FF80015FDE56D902651F8282873900059E0C337
:1010080094024003021157E551D394015003021191
:1010180057E55175F040A4FFAEF090031212001E80
:10102800E0C395455018E55175F040A4FFAEF09027
:10103800031112001EE0F52E752D00021157E5511F
:1010480075F040A4FFAEF090031012001EE0C395A7
:101058004540030210F3E55175F040A4FFAEF0904F
:10106800031112001EE55175F040A4FFAEF0E0FC3C
:1010780090030F12001EECFEE0FFEEC39FFEE55149
:101088008E0475F040A4FFAEF090031012001EE02D
:10109800F40425458C0088F0A4FFAEF0E5518F04D8
:1010A8008E0575F040A4FFAEF090031212001EE505
:1010B8005175F040A4FFAEF0E0FA90031012001E44
:1010C800EAFEE0FFEEC39FFECDCCCD8E0712408531
:1010D800E55175F040A4FFAEF090030F12001EE03A
:1010E8002DFD50010C8C2D8D2E8064E55175F0403E
:1010F800A4FFAEF090030F12001EE55175F040A456
:10110800FFAEF0E0FC90030E12001EECFEE0FFEED6
:10111800C39F8545F0A4FFAEF0E5518F048E057599
:10112800F040A4FFAEF090031012001EE0FECDCCFC
:10113800CD8E07124085E55175F040A4FFAEF090C2
:10114800030E12001EE02DFD50010C8C2D8D2E7506
:101158006D010215FD900059E0C39402400302138B
:101168000B90004FE0D3955150030212B3E551752F
:10117800F040A4FFAEF090031812001EE0C395459E
:101188005018E55175F040A4FFAEF0900317120017
:101198001EE0F52C752B000212B3E55175F040A442
:1011A800FFAEF090031612001EE0C39545400302FF
:1011B800124FE55175F040A4FFAEF09003171200EE
:1011C8001EE55175F040A4FFAEF0E0FC9003151247
:1011D800001EECFEE0FFEEC39FFEE5518E0475F0A5
:1011E80040A4FFAEF090031612001EE0F40425455B
:1011F8008C0088F0A4FFAEF0E5518F048E0575F0E1
:1012080040A4FFAEF090031812001EE55175F0409F
:10121800A4FFAEF0E0FA90031612001EEAFEE0FF0B
:10122800EEC39FFECDCCCD8E07124085E55175F0FB
:1012380040A4FFAEF090031512001EE02DFD5001F2
:101248000C8C2B8D2C8064E55175F040A4FFAEF01A
:1012580090031512001EE55175F040A4FFAEF0E0B2
:10126800FC90031412001EECFEE0FFEEC39F8545C0
:10127800F0A4FFAEF0E5518F048E0575F040A4FF91
:10128800AEF090031612001EE0FECDCCCD8E0712F4
:101298004085E55175F040A4FFAEF09003141200AC
:1012A8001EE02DFD50010C8C2B8D2CE551B4012333
:1012B800E560D39401401CE55604D395514014E5EC
:1012C80045C39405500D90035FE0A829B800069522
:1012D8002A40028003755102E551B5602290004F03
:1012E800E0D395514019E55175F040A4FFAEF09058
:1012F800031712001EE0A823B800069524400280B8
:10130800020560756D020215FD900059E0B4022ACD
:10131800E55175F040A4FFAEF090031712001EE0EF
:10132800F52C752B00E55175F040A4FFAEF0900345
:101338000E12001EE0F52E752D00900059E0B40342
:101348000F900051E0F52C752B00752E00752D00BF
:10135800756D030215FDE55175F040A4FFAEF090E0
:10136800032012001EE0C3955A4003021433900074
:1013780049E07036E551D394014029AE23AF24AC3F
:101388002DAD2EEDD39FEC9E401AE55175F040A48B
:10139800FFAEF090031E12001EE0A829B80005D386
:1013A800952A5002800215518034E551D3940240A9
:1013B80029AE23AF24AC2DAD2EEDD39FEC9E401A61
:1013C800E55175F040A4FFAEF090031E12001EE038
:1013D800A829B80005D3952A500280021551E55175
:1013E800B55237E551C395605030E55604D3955151
:1013F8004028AE23AF24AC2BAD2CEFD39DEE9C4000
:1014080019E55175F040A4FFAEF090031F12001EBD
:10141800E0A829B80006952A400280020551C2902A
:10142800E55165526005C207755A00756D040215CD
:10143800FDE55175F040A4FFAEF090031A12001EAE
:10144800E0B40117E55175F040A4FFAEF090032019
:1014580012001EE0240AC3955A400302150975308C
:1014680064752F00A207B3500B900060E02405C3F9
:1014780095454003021509E55175F040A4FFAEF00B
:1014880090031D12001EE0C395454064E55175F0B8
:1014980040A4FFAEF090031C12001EE55175F04009
:1014A800A4FFAEF0E0FC90031B12001EECFEE0FF70
:1014B800EEC39F8545F0A4FFAEF0E5518F048E057D
:1014C80075F040A4FFAEF090031D12001EE0FECDA3
:1014D800CCCD8E07124085E55175F040A4FFAEF0E3
:1014E80090031B12001EE02DFD50010C8C2F8D3037
:1014F800AE23AF24AC2FAD30EFD39DEE9C4002D28B
:1015080007756D050215FDE551B40109900059E014
:10151800C3940240030215DD900358E0D39545506B
:10152800030215DD900356E0C395455040900357DC
:10153800E0FE900355E0F4042EFE900356E0F40418
:1015480025458E0088F0A4FFAEF0900358E0FC908B
:101558000356E0F4042C8E048F05FF124085900397
:1015680055E02DFD50010C8C2B8D2C802C900355B3
:10157800E0FE900354E0F4042E8545F0A4FFAEF09D
:10158800900356E08E048F05FF124085900354E0C7
:101598002DFD50010C8C2B8D2CE551C395605030DE
:1015A800E55604D395514028AE23AF24AC2BAD2C7F
:1015B800EFD39DEE9C4019E55175F040A4FFAEF0C5
:1015C80090031F12001EE0A829B80006952A4002C1
:1015D8008003755102900049E0B40106E5516401A9
:1015E80060028003755102E55165526005C20775B6
:0515F8005A00756D00B2
:1026510002100302115D02131102135E021439020A
:02266100150F53
:1015FD00900050E02402A823B80007D395244002A0
:10160D00C207900025E0B40109900059E0C394038E
:10161D004003021785900049E060030216D4E5519E
:10162D00D394014034E55175F040A4FFAEF0900322
:10163D001412001EE0A823B8001FD39524401AE50C
:10164D005175F040A4FFAEF090031F12001EE0A8EC
:10165D0029B80005D3952A500280021551E551D3C2
:10166D009401402FE55175F040A4FFAEF0900312A8
:10167D0012001EE0C39545501AE55175F040A4FFC8
:10168D00AEF090031E12001EE0A829B80005D395F8
:10169D002A500280021551E551D394014022E5569E
:1016AD0004C39551501AE55175F040A4FFAEF0906A
:1016BD00031E12001EE0A829B80005D3952A50027A
:1016CD008002155102177AE551D394024034E55149
:1016DD0075F040A4FFAEF090031412001EE0A82395
:1016ED00B8001FD39524401AE55175F040A4FFAE04
:1016FD00F090031F12001EE0A829B80005D3952A0B
:10170D00500280021551E551D39402402FE55175D9
:10171D00F040A4FFAEF090031212001EE0C39545F9
:10172D00501AE55175F040A4FFAEF090031E120063
:10173D001EE0A829B80005D3952A50028002155144
:10174D00E551D394024022E55604C39551501AE554
:10175D005175F040A4FFAEF090031E12001EE0A8DC
:10176D0029B80005D3952A500280021551E551651F
:10177D00526005C207755A00900060E0D395455040
:10178D0009900054E0C395455002C207900059E0FE
:10179D0070030219EAA2A5B34008A2A4B340030244
:1017AD0019D3AE35AF367441D39F749C9E400578E6
:1017BD003512003FAE35AF36EFB48806EEB41302E6
:1017CD0080030219B0A2A55003021873900059E0CE
:1017DD00B4010B90004FE0D395604002056090007E
:1017ED0059E0B40254E55175F040A4FFAEF09003FA
:1017FD002012001EE0C3955A503F90004FE0D39544
:10180D00514021E55604D395514019E55175F040ED
:10181D00A4FFAEF090031412001EE0A823B800063A
:10182D00952440028002055190004FE0F560E5518E
:10183D0065526005C207755A00900059E0B4032641
:10184D0090004FE0D395514008E55604D395515083
:10185D00028002055190004FE0F560E55165526040
:10186D0005C207755A00A2A450030219B090005981
:10187D00E0B4016E900049E07035E551D39401401C
:10188D0029E55175F040A4FFAEF090031E12001E25
:10189D00E0A829B8000FD3952A400A1551755A00B2
:1018AD00855160800385516080037560018033E54B
:1018BD0051D394024029E55175F040A4FFAEF0904C
:1018CD00031E12001EE0A829B8000FD3952A400A66
:1018DD001551755A008551608003855160800375DF
:1018ED006002900059E0D3940150030219A4E55110
:1018FD0075F040A4FFAEF090032012001EE0C395DA
:10190D005A40030219A4900049E07041E551D39467
:10191D00014034E55175F040A4FFAEF09003111273
:10192D00001EE0A823B8001FD39524401AE5517579
:10193D00F040A4FFAEF090031E12001EE0A829B8DF
:10194D000005D3952A500280021551803FE551D3F1
:10195D0094024034E55175F040A4FFAEF0900311B0
:10196D0012001EE0A823B8001FD39524401AE5519C
:10197D0075F040A4FFAEF090031E12001EE0A829E2
:10198D00B80005D3952A500280021551E5516552D4
:10199D006005C207755A00E556B40704055E80035D
:1019AD00755E00E563B4010EAE35AF36EF64407081
:1019BD0005EE649C6002800EA2A54003755801A23D
:1019CD00A44003755802A2A5B3B35006A2A4B3B3A5
:1019DD0040028006753600753500021AD8A2A5B3EF
:1019ED004008A2A4B34003021AC4AE35AF36744109
:1019FD00D39F749C9E4005783512003FAE35AF36AF
:101A0D00EFB48806EEB413028003021AC4A2A540F7
:101A1D006F900068E0605A90004AE0B401079000B2
:101A2D004AE4F0800690004A7401F090004AE0709C
:101A3D0005756003800375600490004AE0B40104ED
:101A4D00D2978002C297E551B4041AE55175F04062
:101A5D00A4FFAEF090031E12001EE0A829B80005E9
:101A6D00D3952A50028008755103C207755A00801C
:101A7D0003756004E556B40704055E8003755E00CA
:101A8D00A2A44033900069E06021900049E0B401C8
:101A9D0007900049E4F080069000497401F0900031
:101AAD0049E0B40104D2A08002C2A0E556B40704F7
:101ABD00055E8003755E00A2A5B3B35006A2A4B364
:101ACD00B340028006753600753500E558655960DE
:101ADD0006900082E06003021C60C29C75140075C4
:101AED001300C2CAE558902663F828287380121295
:101AFD002CE3800D122DBC8008122E958003122F21
:011B0D006E69
:0F266300021AFA021AFC021B01021B06021B0BD1
:101B0E00900029E090007AF0E566900057F0E568C5
:101B1E00900062F0E569900063F0E56A900074F061
:101B2E00E56590007CF0E56790007DF0E56490003F
:101B3E0080F0E563900081F090002AE090013AF089
:101B4E0090002BE090013BF090002CE090013CF0D7
:101B5E00900041E0900090F0900042E0900091F0F3
:101B6E00900043E0900092F0900044E0900093F0DB
:101B7E00900045E0900094F0900046E0900095F0C3
:101B8E00900047E0900096F0900048E0900097F0AB
:101B9E00900033E0900099F0900034E090009AF0BD
:101BAE00900035E090009BF0900036E090009CF0A5
:101BBE007400900082F07446900125F0746F9001CD
:101BCE0026F07472900127F07464900128F074204E
:101BDE00900129F0744190012AF0744F90012BF07E
:101BEE00744490012CF0744590012DF074209001F6
:101BFE002EF0742090012FF07434900130F0745355
:101C0E00900131F07450900132F07444900133F031
:101C1E009003D4E0900414F0743A90074EF074FDE3
:101C2E0090074FF01200C9900004E4F0A3F090006A
:101C3E00067475F0A37430F09000087475F0A374F8
:101C4E0030F0855859D2CA754C00D29C741B900046
:101C5E0023F0E556C394065005E551B55202804E69
:101C6E00C207E55175F040A4FFAEF09003221200BA
:101C7E001EE030E003D38001C39293E55175F0402E
:101C8E00A4FFAEF090032312001EE030E003D380D9
:101C9E0001C39294855152AE29AF2A7405BE00033A
:101CAE009F5007E545D3940550028002D290E55629
:101CBE00D394055003021D85C207E551D39401400C
:101CCE0059E55175F040A4FFAEF090031E12001EB0
:101CDE00E0A829B80007D3952A40021551E55165B1
:101CEE00526035E55175F040A4FFAEF0900322121C
:101CFE00001EE030E003D38001C39293E55175F0EE
:101D0E0040A4FFAEF090032312001EE030E003D398
:101D1E008001C39294855152805DE556B4061A90A7
:101D2E0000ACE030E003D38001C392939000ADE0AD
:101D3E0030E003D38001C39294E556B4071A9000A5
:101D4E00A5E030E003D38001C392939000A6E0306B
:101D5E00E003D38001C39294E556B4081A90009E16
:101D6E00E030E003D38001C3929390009FE030E017
:101D7E0003D38001C39294900072E06058E54575DC
:101D8E00F00284FF7E0090014E12001EE0F55CE52D
:101D9E004775F00A84FF7E0090024E12001EE0F599
:101DAE005DE55C255DD39464400BE55C255DC394D5
:101DBE0064F55C8003755C00E55C75F00284FF7E63
:101DCE00008F5CEFC394335007EF24CDF55C800396
:101DDE00755CFF801CE54575F00284FF7E00900166
:101DEE004E12001EE075F00284FF7E00EF24CDF54A
:101DFE005CE595C3955C4004C2928002D292A20724
:101E0E00B34005E556B407037571CDE595C39571DD
:101E1E004004C2918002D291E543C394064003026E
:101E2E002429A2EDB35003022429C2EDE543600339
:101E3E00021F8B7E017F00E5BE1240A3E5BD2FFF82
:101E4E0050010E900000EEF0A3EFF0900029E0B4E8
:101E5E0001177E0F7FFF900000E0FCA3E0FD120053
:101E6E0003900000EEF0A3EFF0900079E0B4025B77
:101E7E00900000E0FEA3E0FF90000AE0FCA3E0FD6E
:101E8E00EDD39FEC9E400F900000E0F8A3E0900091
:101E9E000AC8F0A3C8F0900000E0FEA3E0FF900097
:101EAE000CE0FCA3E0FDEFD39DEE9C400F900000F4
:101EBE00E0F8A3E090000CC8F0A3C8F0900000E09A
:101ECE00FEA3E0FF74041240958F44900079E070F9
:101EDE0060900000E0FEA3E0FF90000AE0FCA3E0AB
:101EEE00FDEFD39DEE9C400D120003900000EEF02E
:101EFE00A3EFF08007900000E4F0A3F0900000E064
:101F0E00FEA3E0FF74101240A3900026E08E048F13
:101F1E0005FF124085900000ECF0A3EDF07400D3A5
:101F2E009D74019C4008900001E0F54480037544C7
:101F3E00FFE54475F00AA4FFAEF074198E048F0508
:101F4E00FF1240858D45ED2532FFAE3150010E74E6
:101F5E00011240958F45854532753100EFD394625D
:101F6E004003754562900072E06401600690006661
:101F7E00E060028005754301800375BB17E543B42D
:101F8E000102800302207B7E017F00E5BE1240A38A
:101F9E00E5BD2FFF50010E900000EEF0A3EFF09084
:101FAE000072E0B4017EE53445336025AC33AD34C8
:101FBE001DBDFF011C8F028E038C068D07903A6F9C
:101FCE0012002EE493FE740193FFEFC39AEE9B4032
:101FDE0002800578331240CDAE33AF3474B3BE00F9
:101FEE0025D39F4021900000E0FCA3E0FD0FBF0031
:101FFE00010E903A6F12002EE493FE740193FFEDE2
:10200E00C39FEC9E40028005783312003FAE33AF83
:10201E0034E56A1240A374648E048F05FF12408566
:10202E008D478033900066E0602D900000E0FEA3A7
:10203E00E0FFEFD39400EE9408400F900066E0B4FA
:10204E000104C2098002D209800D900066E0B4013D
:10205E0004D2098002C209900072E0640260069008
:10206E000066E0600575BB168003754302E543B458
:10207E00020280030221697E017F00E5BE1240A3A9
:10208E00E5BD2FFF50010E900000EEF0A3EFF09093
:10209E000072E0B4027EE53445336025AC33AD34D6
:1020AE001DBDFF011C8F028E038C068D07903D43D4
:1020BE0012002EE493FE740193FFEFC39AEE9B4041
:1020CE0002800578331240CDAE33AF3474B3BE0008
:1020DE0025D39F4021900000E0FCA3E0FD0FBF0040
:1020EE00010E903D4312002EE493FE740193FFED1A
:1020FE00C39FEC9E40028005783312003FAE33AF93
:10210E0034E56A1240A374648E048F05FF12408575
:10211E008D478033900066E0602D900000E0FEA3B6
:10212E00E0FFEFD39400EE9408400F900066E0B409
:10213E000104C2098002D209800D900066E0B4014C
:10214E0004D2098002C209900072E0700375470044
:10215E00900066E07002C20975BB1FE543B40345EB
:10216E007E017F00E5BE1240A3E5BD2FFF50010E9C
:10217E00900000EEF0A3EFF074091240A374E68E07
:10218E00048F05FF1240858C418D42E54A2DFD508E
:10219E00010C74018C068D071240958E418F42857D
:1021AE00424A75BB19E543B4040280030223117E33
:1021BE00017F00E5BE1240A3E5BD2FFF50010E903A
:1021CE000000EEF0A3EFF074041240958F4BE5641F
:1021DE00B40102800302229E756B00756B00E56BE5
:1021EE00D39407400302228BE56B9000411240BB53
:1021FE00E0D3954B501AE56B9000411240BBE0F4D2
:10220E0004254BFEE56B9000371240BBEEF08017B5
:10221E00E56B9000411240BBE0C3954BFEE56B9021
:10222E0000371240BBEEF0E56BC3940440099000FA
:10223E0084E0C3956B503BE56B6029E56B900037EE
:10224E001240BBFEE0FFEE90003FE0D39F4013E54F
:10225E006B9000371240BBE090003FF0E56B9000B2
:10226E0040F0800E900037E090003FF07400900038
:10227E0040F0786B740126F640030221EC9000408A
:10228E00E0F4042408F556E556D394054002C290B6
:10229E00E564D39401402FE54BD3946E4004D20EE7
:1022AE008002C20E755605E564B40205A20EB34057
:1022BE00028003755607E564B40306A20EB3B3405D
:1022CE00028003755607E55765566008E55104F51B
:1022DE0052855657E556B40708E5B54480F5B580E6
:1022EE0006E5B5547FF5B5E55664066005E556B4CA
:1022FE000808E5B54410F5B58006E5B554EFF5B51B
:10230E0075BB13E543B4050280030224257E017FCD
:10231E0000E5BE1240A3E5BD2FFF50010E90000058
:10232E00EEF0A3EFF074041240958F46E563B4020D
:10233E00028003022422756B00756B00E56BD3944B
:10234E000340030223D9E56B9000331240BBE0D368
:10235E009546501AE56B9000331240BBE0F404250D
:10236E0046FEE56B90002D1240BBEEF08017E56B3C
:10237E009000331240BBE0C39546FEE56B90002DF6
:10238E001240BBEEF0E56B6029E56B90002D12401C
:10239E00BBFEE0FFEE900031E0D39F4013E56B9063
:1023AE00002D1240BBE0900031F0E56B900032F052
:1023BE00800E90002DE0900031F07400900032F00D
:1023CE00786B740126F6400302234A900082E07077
:1023DE0043E52A45296036E558C39403500A900018
:1023EE0032E004C3940340028007900032E004F50B
:1023FE0058E558D39402400A900032E004D3940278
:10240E0050028007900032E004F5588007900032A9
:10241E00E004F55875BB180543D2ECE55ED3940481
:10242E00500302251175CF01C292AE35AF367488B6
:10243E00D39F74139E4005A2A5B34014AE35AF369C
:10244E007488D39F74139E4005A2A4B340028048A3
:10245E00783512003FAE35AF36EFB4883BEEB4138D
:10246E0037A2A5B3500990004FE0D395515002808A
:10247E000405518011A2A5B3500890004FE065519C
:10248E0060028002D207A2A4B35007E551D3940193
:10249E00500280041551C207A2A5B3B35006A2A4E0
:1024AE00B3B340028006753600753500E5516552AE
:1024BE006035E55175F040A4FFAEF0900322120096
:1024CE001EE030E003D38001C39293E55175F040D6
:1024DE00A4FFAEF090032312001EE030E003D38081
:1024EE0001C39294855152A20740057571CD8003A8
:1024FE007571FFE595C395714004C2918002D2912A
:10250E00022433A20DB3500DAE25AF2674E8C39F3F
:10251E0074039E4002800575FFA0D20DAE25AF2636
:10252E00EFD39420EE944E5003022625120481C25E
:10253E008E758D00758B00754C00D28EC20775702E
:10254E0000756F007571CD755104752400752300EB
:10255E00755400755A00C296900059E06004D295E9
:10256E008002C29590004AE0B40104D2978002C264
:10257E0097900049E0B40104D2A08002C2A0A20943
:10258E00B34004D2A28002C2A290006BE060181287
:10259E0036F8A200B34008E5B54408F5B58006E567
:1025AE00B554F7F5B58002C20090006EE0601812C7
:1025BE00384DA202B34008E5B54402F5B58006E5F4
:1025CE00B554FDF5B58006E5B554FDF5B590000E94
:1025DE0074FDF0A374E8F0E543B406037543009070
:1025EE000025E4F0752600752500758D00758B00AD
:1025FE00754C00900024E0C394035008900024E032
:10260E0004F080067403900024F0900024E0B403DC
:10261E0006E5B554FEF5B5AE27AF28EFD39410EE10
:10262E009427401CC2CA75CD0075CC007528007564
:10263E002700D2CA754E00752A00752900755500FF
:03264E00020CC8B3
:1039FF0000000100013201640196019602000212DB
:103A0F0002240200020003000340038003C00400ED
:103A1F000440048004C005000600060006000600EE
:103A2F00060006000600060000FF01310163019544
:103A3F0001FF01FF0211022302FF02FF02FF033FFA
:103A4F00037F03BF03FF043F047F04BF04FF05FF91
:103A5F0006FF06FF06FF06FF06FF06FF06FF06FF2F
:103A6F000FAA0FA50F9F0F9A0F940F8D0F870F801F
:103A7F000F780F710F680F600F570F4E0F450F3BE9
:103A8F000F300F250F1A0F0E0F020EF50EE80EDB7B
:103A9F000ECC0EBE0EAE0E9F0E8E0E7D0E6C0E5AFF
:103AAF000E470E340E200E0C0DF70DE20DCB0DB59B
:103ABF000D9D0D850D6D0D540D3A0D200D050CE965
:103ACF000CCE0CB10C940C760C580C3A0C1B0BFB57
:103ADF000BDB0BBB0B9A0B790B570B350B130AF147
:103AEF000ACE0AAB0A870A640A400A1C09F809D4ED
:103AFF0009B0098C09670943091F08FB08D608B2EA
:103B0F00088E086A0846082307FF07DC07B90796DF
:103B1F0007730751072F070D06EC06CA06AA068979
:103B2F0006690649062A060A05EC05CD05B0059279
:103B3F0005750558053C0520050504EA04CF04B5B5
:103B4F00049C04820469045104390422040B03F415
:103B5F0003DE03C803B2039D038903750361034D9D
:103B6F00033B03280316030402F202E102D102C051
:103B7F0002B002A00291028202730265025702494B
:103B8F00023C022F02220216020901FD01F201E698
:103B9F0001DB01D001C601BB01B101A7019D019459
:103BAF00018B018201790170016801600158015098
:103BBF000148014101390132012B0125011E011874
:103BCF000111010B010500FF00FA0FA60FA00F99BD
:103BDF000F920F8B0F840F7C0F740F6B0F620F58A8
:103BEF000F4E0F430F380F2C0F1F0F120F050EF72D
:103BFF000EE80ED80EC80EB70EA50E930E800E6CE3
:103C0F000E580E420E2C0E150DFD0DE40DCB0DB101
:103C1F000D950D790D5D0D3F0D200D010CE10CC0C3
:103C2F000C9E0C7C0C590C350C100BEA0BC40B9E24
:103C3F000B760B4F0B260AFD0AD40AAA0A800A55E7
:103C4F000A2A09FF09D409A8097C0950092508F98E
:103C5F0008CD08A10875084A081E07F307C8079D75
:103C6F0007730749072006F706CE06A6067E0657F6
:103C7F000630060A05E405BF059B05770554053296
:103C8F00051004EF04CE04AE048F04710453043501
:103C9F00041903FD03E203C703AD0394037B03631E
:103CAF00034B0334031E030802F302DE02CA02B6FB
:103CBF0002A30291027F026D025C024C023C022CB5
:103CCF00021D020E020001F201E401D701CA01BE7A
:103CDF0001B101A6019A018F0185017A0170016678
:103CEF00015D0153014A01410139013101290121CE
:103CFF0001190112010B010400FD00F700F000EAA9
:103D0F0000E400DE00D900D300CE00C900C400BF1C
:103D1F0000BA00B500B100AD00A800A400A0009C3F
:103D2F00009900950091008E008A00870084008121
:043D3F00007E007B87
:10267200751A00751900AE19AF1AAC17AD18EDC373
:102682009FEC9E401674FF12407575CF01781A7444
:102692000126F6500418E436F650DB22900786E451
:1026A200F0A3F0751000750F00751300751400C2C9
:1026B2000FD21022C2AF75D900758F0375B7A575F9
:1026C200B7F190F800E4F0758F0175B7A575B7F111
:1026D200E50890F800F075B7A575B7F190F801E438
:1026E200F075B7A575B7F190079DE090F802F07507
:1026F200B7A575B7F19007A1E090F803F075B7A5FB
:1027020075B7F190079EE090F804F075B7A575B71C
:10271200F190079FE090F805F075B7A575B7F190B5
:1027220007A0E090F806F075B7A575B7F19007A27B
:10273200E090F807F0758F0075D940D2AF2290076C
:1027420088E0B4AB61C2AF75D90075B62275F522C7
:10275200758F0375B7A575B7F1740090F600F07523
:102762008F01750A00750900AE09AF0A7413BE0025
:10277200279F402475B7A575B7F190078912001EEF
:10278200E0FC90F60012001EECF0780A740126F6C6
:10279200500418E436F650D0758F0075F51175B6F1
:1027A2002075D940D2AF22C2AF75D90075F5227516
:1027B2000A00750900AE09AF0A7413BE00229F40D9
:1027C2001F90F60012001EE493FC90078912001E6F
:1027D200ECF0780A740126F6500418E436F650D567
:1027E20075F51175D940D2AF22900788E0B4AA02DC
:1027F2008003022928C2AF75D90075B62275F52269
:10280200758F0375B7A575B7F1740090EE00F0757A
:10281200B7A575B7F1740090F000F075B7A575B75C
:10282200F1740090F200F075B7A575B7F1740090DD
:10283200F400F0758F01750A00750900AE09AF0A40
:1028420074FFC39F74019E402475B7A575B7F190BC
:10285200004E12001EE0FC90EE0012001EECF0781A
:102862000A740126F6500418E436F650CF750A00B1
:10287200750900AE09AF0A74FFC39F74019E40241C
:1028820075B7A575B7F190024E12001EE0FC90F0EC
:102892000012001EECF0780A740126F6500418E4C7
:1028A20036F650CF750A00750900AE09AF0A74FFFB
:1028B200C39F74019E402475B7A575B7F190044E6D
:1028C20012001EE0FC90F20012001EECF0780A7476
:1028D2000126F6500418E436F650CF750A00750941
:1028E20000AE09AF0A74FFC39F74019E402475B7FE
:1028F200A575B7F190064E12001EE0FC90F400128E
:10290200001EECF0780A740126F6500418E436F63C
:1029120050CF758F0075F51175B62075D940D2AFBD
:10292200743A90074EF022900788E0B4AA0280031E
:10293200022A66C2AF75D90075B62275F522758F67
:102942000375B7A575B7F1740090E600F075B7A5E9
:1029520075B7F1740090E800F075B7A575B7F1741A
:102962000090EA00F075B7A575B7F1740090EC001D
:10297200F0758F01750A00750900AE09AF0A74FF80
:10298200C39F74019E402475B7A575B7F190004EA0
:1029920012001EE0FC90E60012001EECF0780A74B1
:1029A2000126F6500418E436F650CF750A00750970
:1029B20000AE09AF0A74FFC39F74019E402475B72D
:1029C200A575B7F190024E12001EE0FC90E80012CD
:1029D200001EECF0780A740126F6500418E436F66C
:1029E20050CF750A00750900AE09AF0A74FFC39F84
:1029F20074019E402475B7A575B7F190044E12007C
:102A02001EE0FC90EA0012001EECF0780A74012627
:102A1200F6500418E436F650CF750A00750900AE78
:102A220009AF0A74FFC39F74019E402475B7A57550
:102A3200B7F190064E12001EE0FC90EC0012001E50
:102A4200ECF0780A740126F6500418E436F650CFFA
:102A5200758F0075F51175B62075D940D2AF743AED
:102A620090074EF022900788E0B4AA028003022B5E
:102A7200A4C2AF75D90075B62275F522758F03759C
:102A8200B7A575B7F1740090DE00F075B7A575B7FC
:102A9200F1740090E000F075B7A575B7F17400907D
:102AA200E200F075B7A575B7F1740090E400F07517
:102AB2008F01750A00750900AE09AF0A74FFC39F42
:102AC20074019E402475B7A575B7F190004E1200AF
:102AD2001EE0FC90DE0012001EECF0780A74012663
:102AE200F6500418E436F650CF750A00750900AEA8
:102AF20009AF0A74FFC39F74019E402475B7A57580
:102B0200B7F190024E12001EE0FC90E00012001E8F
:102B1200ECF0780A740126F6500418E436F650CF29
:102B2200750A00750900AE09AF0A74FFC39F7401EC
:102B32009E402475B7A575B7F190044E12001EE0B1
:102B4200FC90E20012001EECF0780A740126F650A6
:102B52000418E436F650CF750A00750900AE09AFC5
:102B62000A74FFC39F74019E402475B7A575B7F11F
:102B720090064E12001EE0FC90E40012001EECF0E3
:102B8200780A740126F6500418E436F650CF758F91
:102B92000075F51175B62075D940D2AF743A900719
:102BA2004EF022900788E0B4AA028003022CE2C20F
:102BB200AF75D90075B62275F522758F0375B7A565
:102BC20075B7F1740090D600F075B7A575B7F174BA
:102BD2000090D800F075B7A575B7F1740090DA00CF
:102BE200F075B7A575B7F1740090DC00F0758F0130
:102BF200750A00750900AE09AF0A74FFC39F74011C
:102C02009E402475B7A575B7F190004E12001EE0E4
:102C1200FC90D60012001EECF0780A740126F650E1
:102C22000418E436F650CF750A00750900AE09AFF4
:102C32000A74FFC39F74019E402475B7A575B7F14E
:102C420090024E12001EE0FC90D80012001EECF022
:102C5200780A740126F6500418E436F650CF750A45
:102C620000750900AE09AF0A74FFC39F74019E404C
:102C72002475B7A575B7F190044E12001EE0FC90C2
:102C8200DA0012001EECF0780A740126F6500418DD
:102C9200E436F650CF750A00750900AE09AF0A7422
:102CA200FFC39F74019E402475B7A575B7F19006C6
:102CB2004E12001EE0FC90DC0012001EECF0780ABE
:102CC200740126F6500418E436F650CF758F00755D
:102CD200F51175B62075D940D2AF743A90074EF00F
:102CE20022C2AF75D90075F522750A00750900AECA
:102CF20009AF0A74FFC39F74019E401F90EE001239
:102D0200001EE493FC90004E12001EECF0780A7450
:102D12000126F6500418E436F650D4750A007509F7
:102D220000AE09AF0A74FFC39F74019E401F90F06A
:102D32000012001EE493FC90024E12001EECF0788A
:102D42000A740126F6500418E436F650D4750A00C7
:102D5200750900AE09AF0A74FFC39F74019E401F3C
:102D620090F20012001EE493FC90044E12001EEC3E
:102D7200F0780A740126F6500418E436F650D47539
:102D82000A00750900AE09AF0A74FFC39F74019E61
:102D9200401F90F40012001EE493FC90064E1200B5
:102DA2001EECF0780A740126F6500418E436F65048
:102DB200D475F51175D940D2AF22C2AF75D900755D
:102DC200F522750A00750900AE09AF0A74FFC39FA8
:102DD20074019E401F90E60012001EE493FC9000D6
:102DE2004E12001EECF0780A740126F6500418E424
:102DF20036F650D4750A00750900AE09AF0A74FFA1
:102E0200C39F74019E401F90E80012001EE493FCD1
:102E120090024E12001EECF0780A740126F650045D
:102E220018E436F650D4750A00750900AE09AF0AE7
:102E320074FFC39F74019E401F90EA0012001EE4BB
:102E420093FC90044E12001EECF0780A740126F6F0
:102E5200500418E436F650D4750A00750900AE091C
:102E6200AF0A74FFC39F74019E401F90EC001200D2
:102E72001EE493FC90064E12001EECF0780A7401D8
:102E820026F6500418E436F650D475F51175D9407B
:102E9200D2AF22C2AF75D90075F522750A00750945
:102EA20000AE09AF0A74FFC39F74019E401F90DEFB
:102EB2000012001EE493FC90004E12001EECF0780B
:102EC2000A740126F6500418E436F650D4750A0046
:102ED200750900AE09AF0A74FFC39F74019E401FBB
:102EE20090E00012001EE493FC90024E12001EECD1
:102EF200F0780A740126F6500418E436F650D475B8
:102F02000A00750900AE09AF0A74FFC39F74019EDF
:102F1200401F90E20012001EE493FC90044E120047
:102F22001EECF0780A740126F6500418E436F650C6
:102F3200D4750A00750900AE09AF0A74FFC39F7405
:102F4200019E401F90E40012001EE493FC90064E86
:102F520012001EECF0780A740126F6500418E436CA
:102F6200F650D475F51175D940D2AF22C2AF75D9DA
:102F72000075F522750A00750900AE09AF0A74FFE3
:102F8200C39F74019E401F90D60012001EE493FC62
:102F920090004E12001EECF0780A740126F65004DE
:102FA20018E436F650D4750A00750900AE09AF0A66
:102FB20074FFC39F74019E401F90D80012001EE44C
:102FC20093FC90024E12001EECF0780A740126F671
:102FD200500418E436F650D4750A00750900AE099B
:102FE200AF0A74FFC39F74019E401F90DA00120063
:102FF2001EE493FC90044E12001EECF0780A740159
:1030020026F6500418E436F650D4750A0075090005
:10301200AE09AF0A74FFC39F74019E401F90DC008B
:1030220012001EE493FC90064E12001EECF0780A89
:10303200740126F6500418E436F650D475F511756D
:10304200D940D2AF22E51464046006E59964FF60BA
:10305200028031A20F4004D20F8027E51460087469
:10306200E62514900023F0E513600874F025139010
:103072000023F0E514B4010280FE751400751300FC
:10308200C20F8002C20FE5149039A2F82828737586
:103092001400E599B4FF03751301E599B4FE0375B5
:1030A2001302E599B4FD03751303E599B4FC0375A6
:1030B2001304E599B4FA03751305E599B4FB067593
:1030C2001401120481E599B4F906751404120481FD
:1030D200E599D394E54007E599C394F04002801640
:1030E2008599157514027E017F00E515C394E612D9
:1030F20040A38E0D8F0E900786E4F0A3F0E599D3DE
:1031020094C44007E599C394E64002802885991546
:1031120075140374E5C39515F50E750D00AE0DAF6C
:103122000E9039FF12002EE493F8740193900786F3
:10313200C8F0A3C8F0D2990235B6900786E0FEA384
:10314200E0FFEFC39400EE94054009EFD394FFEE45
:1031520094064013900786E0FEA3E0FF90004E1213
:10316200001EE599F0800385996C90078612000E87
:10317200900786E0FEA3E0FFEFB40106EEB407027B
:1031820080030233C690074EE0B43C028003023350
:10319200C6A20AB35005A20BB340030232B9C29CC5
:1031A20090007AE090078CF0900057E090078DF045
:1031B200900062E090078EF0900063E090078FF03D
:1031C200900074E0900790F090007CE0900791F0FE
:1031D20090007DE0900792F0900080E0900793F0DD
:1031E200900081E0900794F090013AE0900795F00A
:1031F20090013BE0900796F090013CE0900797F039
:10320200900090E0900798F0900091E0900799F07C
:10321200900092E090079AF0900093E090079BF064
:10322200900094E090079CF0900095E090079DF04C
:10323200900096E090079EF0900097E090079FF034
:10324200900099E09007A0F090009AE09007A1F01A
:1032520090009BE09007A2F090009CE09007A3F002
:103262007400900082F01200C974AB900788F012CB
:0A327200274074AA900788F0E55881
:0639A20002309102313CED
:10327C009039C3F828287380121227EB800D12297D
:0B328C00298008122A678003122BA57E
:0F39C30002328302328502328A02328F0232943C
:10329700900788E4F090013AE0700C90013BE070F1
:1032A7000690013CE060028004C20A8002D20A0252
:1032B70033BBC29C900078E0900789F090005EE0F5
:1032C70090078AF090005FE090078BF090007AE01B
:1032D70090078CF0900057E090078DF0900062E027
:1032E70090078EF0900063E090078FF0900074E0F5
:1032F700900790F090007CE0900791F090007DE0BF
:10330700900792F0900080E0900793F0900081E0A2
:10331700900794F090013AE0900795F090013BE018
:10332700900796F090013CE0900797F0900090E0AE
:10333700900798F0900091E0900799F0900092E044
:1033470090079AF0900093E090079BF0900094E02C
:1033570090079CF0900095E090079DF0900096E014
:1033670090079EF0900097E090079FF0900099E0FB
:103377009007A0F090009AE09007A1F090009BE0E2
:103387009007A2F090009CE09007A3F074009000D3
:1033970082F074AB900788F012274074AA900788D0
:1033A700F01227EB122929122A67122BA5D29C7536
:1033B70099FB80FED29C7514007513007599FB026A
:1033C70035B6900786E0FEA3E0FFEF4E70068599BD
:1033D70010750F00900786E0FEA3E0FF74016F4EA3
:1033E700701BAC0FAD10AA0DAB0EED2BFBEC3AFA30
:1033F7008A068B0790004E12001EE599F09007860B
:1034070012000E900786E0FEA3E0FF74026F4E7075
:103417000C1200C98515997514007513000235B68D
:10342700900786E0FEA3E0FF90004E12001EE5998C
:10343700F090078612000E900786E0FEA3E0FFAC2F
:103447000DAD0E8F028E038C068D07903A37120052
:103457002EE493F9740193FEEAD39EEB9940098514
:1034670015997514007513000235B6900786E0FEAE
:10347700A3E0FF90004E12001EE599F09007861218
:10348700000E900786E0FEA3E0FFEFB40006EEB45F
:10349700010280030235B690001CE0D394C7400BAD
:1034A70090001CE0C394C8F516801A90001CE0D366
:1034B7009463400B90001CE0C39464F5168006905B
:1034C700001CE0F516E51675F002A4FFAEF08F6B51
:1034D700EF90004E1240BBEFFCE0FDEC9000511264
:1034E70040BBEDFCE0FDEC2DB5160280030235A8CC
:1034F7000FEF90004E1240BBE56BFFE0FCEF900032
:10350700521240BBECFFE0FCEFC39CB516028003F0
:103517000235A8E56B9000501240BBE56BFFE0FC5D
:10352700EF9000531240BBECFFE0FCEF2CB5167197
:10353700E56B9000541240BBE0C3951690079DF0D1
:10354700E56B9000551240BBE0C3951690079EF0BF
:10355700E56B9000581240BBE0C3951690079FF0AB
:10356700E56B9000591240BBE0C395169007A0F099
:10357700E56B90005A1240BBE0C395169007A1F087
:10358700E56B90005B1240BBE0C395169007A2F075
:103597001226B67599F97518647517001226728088
:0F35A700FE7599FF75186475170012267280FE65
:0939A8000233C902342702347213
:1035B60022E5139039B1F82828730236F79007866A
:1035C600E0FEA3E0FF90001212001EE0F5999007BE
:1035D6008612000E900786E0FEA3E0FF74116F4E80
:1035E60070037513000236F78562990236F7900765
:1035F60086E0FEA3E0FF90004E12001EE0F599EF74
:10360600B40107EEB4070375130090078612000E87
:073616000236F7900787E080
:0F39B1000235C00235C30235EE0235F402361975
:10361D009039D2F82828738524990236EC852A9999
:10362D000236EC8544990236EC8547990236EC85D5
:10363D0051990236EC8560990236EC855699023621
:10364D00EC8558990236EC756E00900069E07006B5
:10365D00900068E060028016A2A44006E56E440466
:10366D00F56EA2A54006E56E4402F56E801A900037
:10367D004AE0B40106E56E4410F56E900049E0B4E1
:10368D000106E56E4420F56EA207B34006E56E44D3
:10369D0001F56EA209B34006E56E4408F56E856E20
:1036AD0099803CA210B340077599FAC2108017A2F9
:1036BD000CB3400575990F800B900023E0F59990A0
:1036CD000023E4F0C20C80178542998012854B9936
:0F36DD00800D85469980087599FC800375130050
:1039D20002362402362A02363002363602363C02DB
:1039E200364202364802364E0236540236B00236AB
:0D39F200D50236DA0236DF0236E40236E98D
:0B36EC0090078612000E8003120048B9
:0339C0000236F4D8
:1036F7002290006BE0B4010385241190006BE0B4C5
:103707000203852A1190006BE0B4030385441190EE
:10371700006BE0B4040385471190006BE0B4050328
:1037270085511190006BE0B4060385561190006B2C
:10373700E0B4070385581190006CE0FE90006DE03F
:10374700C39E50030237CE90006BE0D39404402C05
:1037570090006CE0D39511500990006DE0C395116E
:1037670050028002D20090006CE0D395115009906E
:10377700006DE0C395115002C200804990006BE0D4
:10378700B4041890006DE0C395115002D200900068
:103797006CE0D395114002C200802A90006CE0C310
:1037A7009511500990006DE0D3951150028002D217
:1037B7000090006CE0D39511500990006DE0C3951F
:1037C700115002C200807E90006BE0D39404402C1D
:1037D70090006CE0C39511400990006DE0D39511FE
:1037E70040028002C20090006CE0C395114009902E
:1037F700006DE0D395114002D200804990006BE044
:10380700B4041890006CE0C395115002C2009000F8
:103817006DE0D395114002D200802A90006CE0C37E
:103827009511400990006DE0D395114002D20090A8
:10383700006CE0D39511400990006DE0C3951140ED
:10384700028002C2002290006EE0B40103852411B9
:1038570090006EE0B40203852A1190006EE0B40375
:103867000385441190006EE0B4040385471190006E
:103877006EE0B4050385511190006EE0B406038530
:10388700561190006EE0B4070385581190006FE061
:10389700FE900070E0C39E500302392390006EE053
:1038A700D39404402C90006FE0D3951150099000F9
:1038B70070E0C3951150028002D20290006FE0D3EE
:1038C70095115009900070E0C395115002C2028013
:1038D7004990006EE0B40418900070E0C395115051
:1038E70002D20290006FE0D395114002C202802AF3
:1038F70090006FE0C395115009900070E0D39511C7
:1039070050028002D20290006FE0D39511500990C7
:103917000070E0C395115002C202807E90006EE0F5
:10392700D39404402C90006FE0C395114009900098
:1039370070E0D3951140028002C20290006FE0C38D
:1039470095114009900070E0D395114002D2028092
:103957004990006EE0B4041890006FE0C3951150D1
:1039670002C202900070E0D395114002D202802A71
:1039770090006FE0C395114009900070E0D3951156
:103987004002D20290006FE0D39511400990007079
:0B399700E0C3951140028002C2022232
:0940BB002582F5825002058322E2
:10002E00EF2F500205832582F582E5833E2EF58360
:01003E00229F
:08000300C3EF9DFFEE9CFE22FD
:08003F000806B60002180622B3
:0D000E00A3E004F070061240B1E004F022FF
:0840CD000816B6FF02181622C6
:0E409500048007C3CE13CECF13CFD5E0F622A2
:103F4300BC000FBE0008ED8FF084FFADF022E4FE4D
:103F5300FF22BE000DEF60FE54F0606F20E7030206
:103F63003FF9EAC0E0EBC0E078017A0075F001EEBA
:103F730020E710EF25E0FFEE33FE0AC5F023C5F07E
:103F830030E7F0EA5407F9096A7A007B0060010818
:103F9300C3EC9E40167004ED9F4010ED9FFDEC9E18
:103FA300FCE5F0CA4ACA03F5F08005E5F003F5F035
:103FB300C3EE13FEEF13FFD9D77908CACBCAD8D003
:103FC300EAFEEBFFD0E0FBD0E0FA22EC8FF084FCBA
:103FD300ED54F045F0C48FF084FEEDC454F045F089
:103FE300C48FF084FDEEC4FE54F02DFFEE540F3C5D
:103FF300FEADF07C0022790078008FF0EC7E082083
:10400300E70DC3CD33CD33C933C9C833C8DEF0841C
:1040130049F9E5F08FF0BE00E6FD7C00E9FFE8FE1C
:01402300227A
:0E40A300F88FF0A4FFE5F0CE88F0A42EFE22E8
:10407500600D782B02407F007830D8FED5E0F8221D
:10408500EEC0E07E00123F43EFFDEEFCD0E0FE22E5
:03000B000240248C
:03001B0002403F61
:03002B0002405A36
:030000000240C4F7
:0940C40075817275D0000207FD40
:0B001E00E5822FF582E5833EF583228A
:0A40B1000582D582021583158222D4
:10402400C0E0C0F0C083C082C0D075D0001207F2D7
:10403400D0D0D082D083D0F0D0E032C0E0C0F0C085
:1040440083C082C0D075D0001207F5D0D0D082D002
:1040540083D0F0D0E032C0E0C0F0C083C082C0D0D2
:1040640075D0001207F8D0D0D082D083D0F0D0E041
:014074003219
:00000001FF
